:020000040000FA
:04000000A0EF1FF05E
:083F3800000000000000000081
:103F4000720ED36E9B8C240EAC6E190EAF6E900E5B
:103F5000AB6E46D8C10853E1420EAD6E4B0EAD6E4E
:103F6000006A3ED8F86E076E3BD8F76EA96E38D857
:103F7000F66EA86E35D8016E012A00EE09F0F56ED6
:103F80002FD8EC6E012EFBD700661FD007AC03D0F4
:103F9000040E1ED818D007AE04D00C00C40E18D8DA
:103FA00012D0940E15D80A00020E056E00EE0AF02B
:103FB000200E066EEE50F56E0F00062EFBD7840E17
:103FC00007D8052EF5D7A694C9D74E0EAD6EC8D723
:103FD000A66E550EA76EAA0EA76EA682000012004E
:103FE000050E026E036A046A9EAA03D0AE50002634
:103FF0001200042EF9D7032EF6D7022EF3D79CD742
:020000040030CA
:03000100081A1EBC
:020005008181F7
:060008000FC00FE00F40E5
:00000001FF
